:100000000C942A000C9447000C9447000C94470071
:100010000C9447000C9447000C9447000C94470044
:100020000C9447000C9447000C9447000C94470034
:100030000C9447000C9447000C9447000C94470024
:100040000C9447000C9447000C9447000C94470014
:100050000C94470011241FBECFE5D4E0DEBFCDBF16
:1000600010E0A0E6B0E0EEE1F2E002C005900D92F3
:10007000A237B107D9F710E0A2E7B0E001C01D92A6
:10008000A237B107E1F70E9484000C940E010C9492
:100090000000AC01892B59F020E030E08AEF90E0BD
:1000A0000197F1F72F5F3F4F24173507B9F70895F0
:1000B000BB9ABC98BD9A8A98BA9AA19AA39A0895B5
:1000C000C29AC39AC59880B386B3A99A0895C59871
:1000D000C29820E0C598C598992314F4C39A01C02A
:1000E000C398C59AC59A2F5F203119F0880F991FC0
:1000F000F1CFC598C29A08958299FECF90E08050C2
:1001000098440E9467000895CF92DF92EF92FF9289
:100110000F931F93CF93DF930E9458000E946000BB
:10012000AB9A84E690E00E94490087EE90E80E9436
:10013000670089E392E80E94670080E496EA0E94E3
:10014000670083E296EC0E94670080E298E90E94D3
:10015000670000E00F2EF0E6CF2EF0E0DF2EF02D4E
:10016000EE24FF246894E4F8EC0CFD1CAB9A80E0CC
:1001700090E00E94670089E392E80E94670010E027
:100180008AEA0E947C001F5F1330D1F78DE20E9443
:100190007C0084ED0E947C00E60110E088810E94D2
:1001A0007C008991180FCE15DF05C1F7812F0E94C1
:1001B0007C008AEA0E947C008AEA0E947C0081E03E
:1001C00092E80E946700AB9884EF91E00E9449009A
:1001D0000F5F802F64E60E940201805D80936D00B6
:1001E000802F0E940201292F892F6AE00E940201BC
:1001F000805D80936E00822F0E940201905D90933B
:100200006F00B4CF991B79E004C0991F961708F0CE
:0E021000961B881F7A95C9F780950895FFCF39
:10021E000A0D41546D65676131360A0D202D2D2D65
:02022E000000CE
:00000001FF
